:03000000024EAD00
:0C4EAD0078FFE4F6D8FD758177024EF422
:10155D0020000A3C2E2E2E3E004950436F6E6E65C4
:10156D0063745245510A004950436F6E6E65637442
:10157D00000A49504E6F41434B210A003E432C5601
:10158D002C43432CC0E4E0EFF2E5F020D1E8EDEA86
:10159D00EEEC49500A003E432C4D41432C25303290
:1015AD0062583A25303262583A25303262583A251F
:1015BD00303262583A25303262583A25303262580C
:1015CD002C4D414320E0E4F0E5F10A003E432C565A
:1015DD0045522C20332E3220EEF220257320257318
:1015ED002CC2E5F0F1E8FF20495020ECEEE4F3EBDE
:1015FD00FF0A004E6F762032322032303038003004
:10160D00383A33333A3236003E432C4C442C505248
:10161D004F473A202020202020202020202020204D
:10162D0020202020202020202020202020202020AD
:10163D00202020202020202020202020202020209D
:10164D00202020202020202020202020202020208D
:10165D0020202020202020202CC4E0F2E020EFF0DC
:10166D00EEF8E8E2EAE828F4E0E9EB290A003E2A80
:10167D002C312CCEF1EDEEE2EDFBE520EFE0F0E0CC
:10168D00ECE5F2F0FB20F1E5F2E5E2EEE3EE20E829
:10169D00EDF2E5F0F4E5E9F1E00A003E412C4130D0
:1016AD00312C2562752E2562752E2562752E2562CB
:1016BD00752C495020E0E4F0E5F120E0E4E0EFF294
:1016CD00E5F0E00A003E412C4130322C2562752EAA
:1016DD002562752E2562752E2562752C495020E0E8
:1016ED00E4F0E5F120EEF1ED2E20F1E5F0E2E5F08C
:1016FD00E00A003E412C4130332C2562752E2562C7
:10170D00752E2562752E2562752C495020E0E4F06A
:10171D00E5F120F0E5E72E20F1E5F0E2E5F0E00A55
:10172D00003E412C4130342C2562752E2562752EDC
:10173D002562752E2562752CCCE0F1EAE020F1E5ED
:10174D00F2E80A003E412C4130352C2562752E25DC
:10175D0062752E2562752E2562752CD8EBFEE70A73
:10176D00003E2A2C312CC4EEEF2E20EFE0F0E0EC01
:10177D00E5F2F0FB20F1E5F2E5E2EEE3EE20E8ED37
:10178D00F2E5F0F4E5E9F1E00A003E422C53303188
:10179D002C2562752CC6E4E0F2FC20E7E0EFF0EEBC
:1017AD00F1E020F1EEE5E4E8EDE5EDE8FF20EEF205
:1017BD0020F1E5F0E2E5F0E00A003E422C53303234
:1017CD002C2562752CCEE1ECE5ED20F120F1E5F054
:1017DD00E2E5F0EEEC20E1E5E720EAE2E8F2E0ED0B
:1017ED00F6E8E90A003E422C5330332C2562752C65
:1017FD00CFE5F0E5E7E0EFF3F1EA20EFF0E820EFD9
:10180D00EEF2E5F0E520F1E2FFE7E820F120F1E569
:10181D00F0E2E5F0EEEC0A003E422C5330352C257B
:10182D0062752CCAE0EDE0EB20F8E8F0EEEAEEE2AE
:10183D00E5F8E0F2E5EBFCEDEEE3EE20EEE1ECE5B4
:10184D00EDE00A003E532C5330362C2530326258D1
:10185D002530326258253032625825303262582593
:10186D003032625825303262582C4D414320E0E42D
:10187D00F0E5F120F8E8F0EEEAEEE2E5F8E0F2E569
:10188D00EBFCEDEEE3EE20EEE1ECE5EDE00A003EE3
:10189D00454E440A000A44756D70582020202020C2
:1018AD003030203031203032203033203034203071
:1018BD003520303620303720303820303920304137
:1018CD002030422030432030442030452030460027
:1018DD000A3A003A20000A000A44756D704420202F
:1018ED002020203030203031203032203033203055
:1018FD003420303520303620303720303820303904
:10190D0020304120304220304320304420304520CB
:10191D00304600457272206B657900526420656512
:10192D0070726F6D0A005264204D454D0A0052646D
:10193D0020436F64650A00577269746520436F64B4
:10194D00650A0044656275674950204F4E0A004490
:10195D00656275674950204F46460A0044656275B9
:10196D006755736572204F6E0A0044656275675541
:10197D00736572204F46460A0044656275674D7364
:10198D0067204F6E0A0044656275674D7367204F7F
:10199D0046460A00436F6E666967206C6F636B2164
:1019AD000A00577220656570726F6D0A00205361D1
:1019BD00766520656570726F6D210A004572722023
:1019CD004D414321004C6F61643E3E002A003C4175
:1019DD0030313D003C4130323D003C4130333D0023
:1019ED003C4130343D003C4130353D003C21003C14
:1019FD005330313D003C5330323D003C5330333D8C
:0D1A0D00003C5330353D003C5330363D0069
:06594A000174000172006F
:10590D00C28E438910758BFF758DB7D2ABD28E22A7
:03001B00024E1D75
:104E1D00C0E0C083C082C0D0C28E758BFF758DB7C8
:104E2D00201A0675A61E75A6E10572D216E57460E8
:104E3D00020574E573D39401400215730577E57788
:104E4D00540F7048D222E577543F7012D2149070EF
:104E5D0005E0600A04F0E0D394B44002D21A9070D9
:104E6D0000E0600204F0906A7EE0600214F0907041
:104E7D0006E0D394014003E014F03019020575E506
:104E8D0076D394644004D21A80020576E571D394EA
:104E9D000140021571D28ED0D0D082D083D0E032B5
:100EFD00C291C290D2B5C21F7D027C007F071258ED
:100F0D00D68F27E527646060097D017F60125871D7
:100F1D00D21FE4FDFC7F0B1258D68F27E52730E654
:100F2D00097D04E4FF125895D21F7D017C007F07D7
:100F3D001258D68F27E5277008FD7FFF125871D202
:100F4D001F301F03126000C288C2A8C2AA75890093
:100F5D00125259906CB8E0B4FA06A3E064CE607BEF
:100F6D00E4F52774B02527F582E4346CF583E4F0BD
:100F7D000527E527B443EC906CB874FAF0A374CE52
:100F8D00F0A374CCF0906CBE740AF0E4A3F0A3044B
:100F9D00F0A3F0906CB474FFF0A3F0A3F0E4A3F011
:100FAD00906CCF740AF0E4F527E5272401FFE433B4
:100FBD00FE74B02527F582E4346CF583E0FD1258FC
:100FCD004D0527E527C3944340DFE4F5A775A61E1D
:100FDD0075A6E1907FF0F0A3F080FE906CC37403D2
:100FED00F0A374CCF0E4906CC2F0124B52C2B51267
:100FFD0047CBC21A1255AAD21FC221C220906EF041
:10100D007408F0906C2E7424F0E4A3F0906CB8E0AA
:10101D00906C30F0906CB9E0906C31F0906CBAE05F
:10102D00906C32F0906CBBE0906C33F0906CBCE047
:10103D00906C34F0906CBDE0906C35F0757301E4FC
:10104D00906EF1F0C21BC21CC21DC21E125826208A
:10105D001F19AF277E007D0312499CE4FF124C1C23
:10106D007E157F5DE4FBFDFC1243DE907005E060B4
:10107D00037401F0E4906A7EF0F575906EEFF0F573
:10108D007612590D75A70775A61E75A6E1D2AFE4A8
:10109D00F576906A7EE07003122353907006E0B4EB
:1010AD0001119080007410F0E4907006F0D21FC210
:1010BD0020C221908008E0F52730E405D21B741082
:1010CD00F0E52730E508D21D9080087420F0E52763
:1010DD0030E608D21C9080087440F0E575C3940387
:1010ED004019908002E4F0908001F0908000F0E5CE
:1010FD007594064006E4F5751255AA9080A0E0702F
:10110D00031252D79080B8E070031253519080D0E3
:10111D00E0700312554E908000E07013301B1012DA
:10112D0044E5906CABEFF0D3940040031200269091
:10113D008002E07006908000E06005D21902109CDC
:10114D00C219E4F575906A7EE0600302109C201FC1
:10115D0012906EF2E0600C7E157F5F1248B4E49041
:10116D006EF2F0301D12123C56906CABEFF0D39432
:10117D00004005E0FF12591D201C03021305123A11
:10118D00CF906CABEFF0700302109C906CEFE054BD
:10119D00BF247F700302126E1470030212462402E4
:1011AD0060030212A7201F077E157F661248B42028
:1011BD002303021305906CC7E07006906CCBE060C2
:1011CD0067906FFCE0FF906CC7E0B50724906FFD52
:1011DD00E0FE906CC8E0B50618906FFEE0FE906CD6
:1011ED00C9E0B5060C906FFFE0FE906CCAE06E6032
:1011FD0037906CCBE06F6003021305906FFDE0FF3D
:10120D00906CCCE06F6003021305906FFEE0FF90D1
:10121D006CCDE06F6003021305906FFFE0FF906CE3
:10122D00CEE06F6003021305C217906EF17401F0EA
:10123D00120021757301021305907005E0600374AF
:10124D0001F0906FF4E0FF906CF1E06F600302131A
:10125D0005906FF4E004F0E4F573906EEFF0021377
:10126D0005301703021305906CBEE0700302109C4D
:10127D00906CCF740AF0125951D217E4F573906E39
:10128D00EFF090700004F0E4906FF3F0A3F0201FE6
:10129D00677E157F741248B4805E907005E0600320
:1012AD007401F0301752906CEFE020E74B906CF129
:1012BD00E0FF906FF3E0FE6F600D906FFBE0700745
:1012CD00EE146F70338013906FF3E004F0906CABFD
:1012DD00E0FFD39404400312569290697A7482F021
:1012ED00A37401F0906CF1E090697CF07E697F7AD7
:1012FD007D03124FC002109C20170302141DE573CD
:10130D007068125772EF60237E6D7FEF906DF0E085
:10131D002404FD124FC0906FFBE07009906CCFE07C
:10132D00F57302109CE4F57302109C907000E0D3ED
:10133D00943C4036906FFBE0703090700004F012DA
:10134D005937E4906DEFF0A37412F0906FF4E090C4
:10135D006DF1F0A374FDF0906A7F63A201906DF3BF
:10136D0063A2017F12123649809E12592C8F27E5F8
:10137D0027B4011590697A7483F0E4A3F07E697F38
:10138D007A7D02124FC002109CE527D39401401CB8
:10139D0090697A7483F0A37401F0E52724FEA3F01D
:1013AD007E697F7A7D03124FC002109CE573640144
:1013BD00600302109C906EEFE004F0201F077E1575
:1013CD007F7E1248B4906CCFE0C394C85004E024E3
:1013DD0032F0906EEFE0C39405400DC217E4906EAD
:1013ED00F1F012002102109C7C6F7DFC906CC3E02B
:1013FD00FAA3E0FB7F021251517E6D7FEF906DF0ED
:10140D00E02404FD124FC0906CCFE0F57302109CE8
:10141D00E5736401600302109C906EF1E014604668
:10142D0024FE6042147003021510240460030210A0
:10143D009CE4F575202313906EF17404F0906EEF1B
:10144D00E05401F075730102109C9080027410F04D
:10145D00E4906EF1F0906EEF04F07573FA906FFCFE
:10146D0074FFF002109C906FFCE070030214FA9070
:10147D006DEF7480F0906DF17401F0E4A3F0A304AE
:10148D00F0A37430F0A3747BF0E4F52774F62527F0
:10149D00F582E4346DF583747DF074F72527F582BC
:1014AD00E4346DF583E4F0E5272407906DF0F07CCE
:1014BD006F7DFC906CC3E0FAA3E0FB7F02125151EB
:1014CD007E6D7FEFE5272409FD124FC0906FFBE085
:1014DD00601B125951D217E4F573906EEFF09070B6
:1014ED000004F0E4906FF3F0A3F002109C3023079A
:1014FD00E4906EF1F08006906EF17404F07573FA5D
:10150D0002109C9080027410F0757305906EEFE0E0
:10151D006401FFF0906EF17401F0EF7019906CCBD7
:10152D00E06013FCA3E0FDA3E0FEA3E0FF906FFCE1
:10153D00122C1D02109C906CC7E0FCA3E0FDA3E0F3
:0F154D00FEA3E0FF906FFC122C1D02109C80FE8D
:01155C00226C
:10002600906CF0E0B444047F0180027F00906CEF96
:10003600E0B447047E0180027E00EE5F604A906C69
:10004600B8E0906CF1F0906CB9E0906CF2F0906CC6
:10005600BAE0906CF3F0906CBBE0906CF4F0906CAE
:10006600BCE0906CF5F0906CBDE0906CF6F0906C96
:10007600F07452F0906C2863A2019080A863A201EC
:100086007F0612364902087B906CABE0C394085099
:1000960003020884906CB8E0FF906CF1E06F600397
:1000A600020884906CB9E0FF906CF2E06F60030286
:1000B6000884906CBAE0FF906CF3E06F600302086E
:1000C60084906CBBE0FF906CF4E06F6003020884E0
:1000D600906CBCE0FF906CF5E06F600302088490C2
:1000E6006CBDE0FF906CF6E06F6003020884906CD4
:1000F600F0E0B44415906C28E0B4FF0E63A20190C2
:1001060080A863A2017F06123649907005E060035D
:100116007401F09070067464F0906CF07452F09074
:100126006CEFE0646D60030202857BFF7A157989C6
:100136001227997BFF7A1579A3906CB8E0F530A366
:10014600E0F531A3E0F532A3E0F533A3E0F534A3FF
:10015600E0F5351227997530FF7531167532007541
:1001660033FF75341675350C7BFF7A1579D912274E
:10017600997BFF7A1679151227997BFF7A16797B78
:100186001227997BFF7A1679A8906CBEE0F530A30A
:10019600E0F531A3E0F532A3E0F5331227997BFFB2
:1001A6007A1679D2906CC7E0F530A3E0F531A3E07A
:1001B600F532A3E0F5331227997BFF7A1779009081
:1001C6006CCBE0F530A3E0F531A3E0F532A3E0F522
:1001D600331227997BFF7A17792E906CB4E0F530AD
:1001E600A3E0F531A3E0F532A3E0F5331227997BBE
:1001F600FF7A177951906CB0E0F530A3E0F531A3A2
:10020600E0F532A3E0F5331227997BFF7A17796E72
:100216001227997BFF7A177997A223E433F53012D8
:1002260027997BFF7A1779C7906FFBE0F530122785
:10023600997BFF7A1779F2907005E0F530122799CD
:100246007BFF7A187925A215E433F5301227997BBE
:10025600FF7A187951906FF5E0F530A3E0F531A3F8
:10026600E0F532A3E0F533A3E0F534A3E0F535126B
:100276002799123F227BFF7A18799C1227992290A0
:100286006CEFE0644C70737E187FA2FBFDFC12439A
:10029600DE906CF7E0F528A3E0F529E4F52BE528D8
:1002A600906CF9F0A3E529F07E187FDD7C6C7DF972
:1002B6007B021243DEE4F52A852982852883E0FF46
:1002C60074F9252AF582E4346CF583EFF00529E507
:1002D6002970020528052AE52AB410DC7E187FE07D
:1002E6007C6C7DF97B101243DE052BE52BC3941045
:1002F60040AC7E187FE31248B422906CEFE0646C49
:100306007060F52C7E187FE5FBFDFC1243DEE4F5FC
:100316002BE4906CF9F0A3E52CF07E187FDD7C6C65
:100326007DF97B021243DEE4F52AA82CE6FF74F978
:10033600252AF582E4346CF583EFF0052C052AE5D1
:100346002AB410E67E187FE07C6C7DF97B101243A0
:10035600DE052BE52BC3940840B77E187FE31248D1
:10036600B422906CEFE0644B7061F52A74E1252AA3
:10037600F582E4346CF583E0603274E1252AF58277
:10038600E4346CF583E0F4602374E1252AF582E415
:10039600346CF583E0FF74F7252AF582E4346CF5B6
:1003A60083E0B50710052AE52AB408C0906A7E7472
:1003B60032F002087B906CEF7421F0301F030208C4
:1003C6007B7E197F201248B402087B906CEFE0B464
:1003D600521A201F077E197F281248B4906CEF74BA
:1003E60072F07E6C7FEF7D08124F3922906CEFE041
:1003F60064497045201F077E197F331248B4906CFC
:10040600F7E0F528A3E0F529E4F52A852982852871
:1004160083E0FF74F9252AF582E4346CF583EFF066
:100426000529E52970020528052AE52AB480DC7E1F
:100436006C7FEF7D8A124F3922906CEFE064437037
:1004460046201F077E197F3B1248B4906CF7E0F5F3
:1004560028A3E0F529E4F52A852982852883E493F3
:10046600FF74F9252AF582E4346CF583EFF005294B
:10047600E52970020528052AE52AB480DB7E6C7F13
:10048600EF7D8A124F3922906CEFE0645A70532048
:100496001F077E197F441248B4906CF7E0F528A335
:1004A600E0F5297C6C7DF97B80AF29AE2812573E9A
:1004B600E4F52A852982852883E493FF74F9252AA1
:1004C600F582E4346CF583EFF00529E52970020521
:1004D60028052AE52AB480DB7E6C7FEF7D8A124FE1
:1004E6003922906CEFE064446003020579906CF762
:1004F600E0FF6444700302087BEFB4310CC21F7E38
:10050600197F501248B402087B906CF7E0B4300CA7
:10051600D21F7E197F5C1248B402087B906CF7E00C
:10052600B4320CD2207E197F691248B402087B903F
:100536006CF7E0B4330CC2207E197F771248B40200
:10054600087B906CF7E0B4340CD2217E197F8612BA
:1005560048B402087B906CF7E0B4350CC2217E19D2
:100566007F931248B402087B906CF7E0FF12001EDE
:1005760002087B906A7EE07013201F077E197FA118
:100586001248B4906CEF7421F002087B906A7E7476
:1005960032F0906CEFE0FFB45104C2AF80FEEF641E
:1005A600577045201F077E197FAF1248B4906CF82C
:1005B600E0906CABF0E4F52A906CABE0FFE52AC363
:1005C6009F400302087B74F9252AF582E4346CF512
:1005D60083E0FF906CF7E0252A2427F582E4346B4C
:1005E600F583EFF0052A80D0906CEFE0645360034A
:1005F60002069C201F077E197FBA1248B4906CB879
:10060600E0FF906B30E06F703C906CB9E0FF906B50
:1006160031E06F7030906CBAE0FF906B32E0B50756
:1006260024906CBBE0FF906B33E0B50718906CBC70
:10063600E0FF906B34E0B5070C906CBDE0FF906B6B
:1006460035E06F6016906CEF7421F0301F030208DE
:100656007B7E197FC91248B402087BE4F52AE4F5CB
:1006660076AF2AFE7427252AF582E4346BF583E0FB
:10067600FD12584D052AE52AC394FE40E1C2AFE4B7
:10068600907FF0F0A3F0907FFD74AAF0A374FFF0C2
:10069600A37455F080FE906CEFE0644F704C906C44
:1006A600F7E0F528A3E0F529E5294528700A201F7B
:1006B600077E197FD21248B4201F077E197FD912F0
:1006C60048B4E4F52A74F9252AF582E4346CF583F6
:1006D600E0852982852883F00529E5297002052809
:1006E600052AE52AB480DE02087B906CEFE0FFB4B1
:1006F6004521906CF7E0FDA3E0907FF0CDF0A3EDEF
:10070600F0C2AF907FFD74AAF0A374FFF0A37455F6
:10071600F080FEEF64656003020884906CF7E0FFEA
:10072600A3E0907FF0CFF0A3EFF0E4F528F529D30E
:10073600907FF1E09529907FF0E095284020E4F540
:10074600762529FFE5283401FE852982852883E060
:10075600FD12584D0529E5297002052880D17E191C
:100766007FDB125047EF4E6020120003906CBEEF05
:10077600F0120003906CBFEFF0120003906CC0EF14
:10078600F0120003906CC1EFF07E197FE112504722
:10079600EF4E6020120003906CC7EFF0120003903A
:1007A6006CC8EFF0120003906CC9EFF012000390D2
:1007B6006CCAEFF07E197FE7125047EF4E602012A9
:1007C6000003906CCBEFF0120003906CCCEFF012AC
:1007D6000003906CCDEFF0120003906CCEEFF07E2C
:1007E600197FED125047EF4E6020120003906CB453
:1007F600EFF0120003906CB5EFF0120003906CB6A8
:10080600EFF0120003906CB7EFF07E197FF31250F1
:1008160047EF4E6020120003906CB0EFF012000319
:10082600906CB1EFF0120003906CB2EFF01200037F
:10083600906CB3EFF0E4F52AE4F576E52A2401FF9F
:10084600E433FE74B0252AF582E4346CF583E0FDCA
:1008560012584D052AE52AC3944340DCC2AFE49002
:100866007FF0F0A3F0907FFD74AAF0A374FFF0A3CD
:0E0876007455F080FE7E6C7FEF7D08124F39C6
:010884002251
:1056D000AE07EEC39430400BEED394395005EE2460
:1056E000D0FF22EEC39461400BEED394665005EEDA
:1056F00024A9FF22EEC39441400BEED394465005FB
:08570000EE24C9FF22AF0622CE
:1058F300906C27E004F07006906C26E004F0906C46
:0A59030026E0FEA3E0FF1258B922CF
:100003001258F31256D0EFC454F0FEC0061258F340
:080013001256D0D0E02FFF22AD
:1054F100E490725FF01258F3907260EFF0C3943051
:105501004018E0FFD39439501190725FE0247FF589
:1055110082E4346AF583EFF0801190725FE0247FBA
:10552100F582E4346AF583E4F0800C90725FE00464
:10553100F0E0D3940840BE752B00752C00752D004A
:0C554100E4F52E7B017A6A797F12392B89
:01554D00223B
:045047008E2D8F2EED
:10504B00906C26E4F0A374FFF01258F3EF606EF44B
:10505B00606B852E82852D83E493B507EC752F014C
:10506B00E52E252FF582E4352DF583E4936025900D
:10507B006C27E0252FFF906C26E03400FE1258B908
:10508B00E52E252FF582E4352DF583E493B5070442
:10509B00052F80CCE52E252FF582E4352DF583E405
:1050AB009370A6E52F24FFFFE434FFFE906C27E0FE
:1050BB002FF0906C26E03EF07E007F0122E4FEFF95
:0150CB0022C2
:104B52007E197FF9125047EF4E70037F01227E19B2
:104B62007FFC125047EF4E600C1258F3EF24D02412
:104B7200FF92238002D2237E1A7F02125047EF4E09
:104B8200600C1258F3EF24D0906FFBF08005E49094
:104B92006FFBF07E1A7F08125047EF4E600C1258DE
:104BA200F3EF24D0907005F08005E4907005F07E5C
:104BB2001A7F0E125047EF4E600C1258F3EF24D0BA
:104BC20024FF92158002C215906CB863A201906F07
:104BD200F563A2017F0612364930153B7E1A7F1417
:104BE200125047EF4E6030120003906FF5EFF01253
:104BF2000003906FF6EFF0120003906FF7EFF012E0
:104C02000003906FF8EFF0120003906FF9EFF012CB
:0A4C12000003906FFAEFF07F00221C
:10560400906EF0E0C3947C503D906EF0E0FE04F0A8
:10561400742E2EF582E4346CF583EFF0BF0A2790E4
:105624006EF0E0FF04F0742E2FF582E4346CF58301
:10563400E4F0906EF0E0FF1250CC906EF07408F03D
:07564400906C2FE004F0223E
:1055AA009080007480F0906CB063A201F583F5825C
:1055BA0063A2017F08123649906CB863A2019080F9
:1055CA008863A2017F0A1236499080927407F0A379
:1055DA0074D0F0A37406F0906CC2E0FF9080B1F032
:1055EA009080E1EFF09080957455F0A3F0908000E0
:0A55FA007401F090800974F0F022B3
:1052D700908009E04410F09080A0E0706C9080A16D
:1052E7007482F09080A874FFF0A3F0A3F0A3F07F7E
:1052F700039080AEEFF07FCBA3EFF07F039080ACFD
:10530700EFF0A374CBF09080007402F09072391222
:105317002C2900000000907239E0908040F09072D4
:105327003AE0908041F090723BE0908042F09072BA
:105337003CE0908043F0A3E4F0A3F0A3F0A3F09047
:095347008018F0A3F0A3F0A3F01C
:01535000223A
:10554E00908009E04440F09080D17482F07F039007
:10555E0080DEEFF0A374CCF09080027402F09072B3
:10556E003D122C290000000090723DE0908058F012
:10557E0090723EE0908059F090723FE090805AF029
:10558E00907240E090805BF0A3E4F0A3F0A3F0A350
:0B559E00F0908030F0A3F0A3F0A3F029
:0155A90022DF
:10535100908009E04420F09080B8E0706C9080B9B2
:105361007482F07F039080C6EFF07FCDA3EFF07FD2
:10537100039080C4EFF0A374CDF09080C074FFF06F
:10538100A3F0A3F0A3F09080017402F09072411297
:105391002C2900000000907241E090804CF0907246
:1053A10042E090804DF0907243E090804EF0907218
:1053B10044E090804FF0A3E4F0A3F0A3F0A3F090B9
:0953C1008024F0A3F0A3F0A3F096
:0153CA0022C0
:105151008C288D29A907EAFDE975F018A424ACFF74
:10516100E5F034808F82F583EDF0EBFDE975F01801
:10517100A4FFAEF024ACFBEE34808B82F583A3ED6B
:10518100F08529828C83E0FDEF24A8FFEE3480FEB8
:105191008F82F583EDF08529828C83A3E08F828E47
:1051A10083A3F0852982852883A3A3E0FDE975F017
:1051B10018A424A8FFE5F03480FE8F82F583A3A311
:1051C100EDF08529828C83A3A3A3E08F828E83A334
:0451D100A3A3F02282
:064F39008D2DAB07AA0656
:104F3F00908000E030E507906EF27401F0229072DD
:104F4F0039E0FCA3E0FDA3E0FEA3E0F5318E308D48
:104F5F002F8C2EAE02AF038E838F8263A201E530BA
:104F6F00540744C0F58385318263A201AF2D1236F9
:104F7F00BBE4FCFDFEE531252DF531EE3530F53086
:104F8F00ED352FF52FEC352EF52E908040E52EF0D8
:104F9F00A3E52FF0A3E530F0A3E531F09080007486
:104FAF0020F0AF31AE30AD2FAC2E907239122C1DD8
:014FBF0022CF
:064FC0008D28AB07AA06D4
:104FC600908002E030E507906EF27403F022907252
:104FD6003DE0FCA3E0FDA3E0FEA3E0F52C8E2B8DC7
:104FE6002A8C29AE02AF038E838F8263A201E52B42
:104FF600540744D0F583852C8263A201AF2812366C
:10500600BBE4FCFDFEE52C2528F52CEE352BF52B17
:10501600ED352AF52AEC3529F529908058E529F051
:10502600A3E52AF0A3E52BF0A3E52CF0908002740B
:1050360020F0AF2CAE2BAD2AAC2990723D122C1D60
:015046002247
:024C1C008F29DE
:104C1E00908001E030E509906EF27402F07F002280
:104C2E00907241E0FCA3E0FDA3E0FEA3E0F52D8E23
:104C3E002C8D2B8C2A906FF563A201E52C54074422
:104C4E00C8F583852D8263A2017F061236D1E52D2C
:104C5E002406F52DE4352CF52CE4352BF52BE43517
:104C6E002AF52A906EF363A201E52C540744C8F589
:104C7E0083852D8263A201AF291236D1E4FCFDFE9D
:104C8E00E52D2529F52DEE352CF52CED352BF52BB7
:104C9E00EC352AF52A90804CE52AF0A3E52BF0A3FB
:104CAE00E52CF0A3E52DF09080017420F0AF2DAE31
:0D4CBE002CAD2BAC2A907241122C1DAF2999
:014CCB0022C6
:1044E5009081E0E0F52805280528052805280528F8
:1044F50005280528052805280528908010E0F52BB6
:10450500A3E0F52CA3E0F52DA3E0F52E9081E1E0E5
:10451500F52805280528052805280528052805283E
:10452500052805280528908014E0F52FA3E0F5302F
:10453500A3E0F531A3E0F532E531B52D08E532B557
:104545002E037F0022E4F528E531540744E0F58386
:1045550085328263A201906CEF63A2017F08123756
:1045650001906CF163A201906C2863A2017F061291
:104575003649906CEFE0F529A3E0F52AE4F528909B
:104585006CEFE0702AA3E024F8F528E531540744E0
:10459500E0F58385328274082582F582E43583F55A
:1045A5008363A201906CEF63A201AF28123701AEBD
:1045B50029E4FCFDE532252AF532E5313EF531EDFC
:1045C5003530F530EC352FF52F908014E52FF0A31D
:1045D500E530F0A3E531F0A3E532F09080007440BA
:0345E500F0AF280C
:0145E80022B0
:103ACF009081E6E0F5280528052805280528052812
:103ADF0005280528052805280528908028E0F52BBE
:103AEF00A3E0F52CA3E0F52DA3E0F52E9081E7E000
:103AFF00F52805280528052805280528052805285F
:103B0F0005280528052890802CE0F52FA3E0F53037
:103B1F00A3E0F531A3E0F532E4F528E531B52D0A40
:103B2F00E532B52E05C21C023C3BE531540744F08B
:103B3F00F58385328263A201906CEF63A2017F0847
:103B4F00123701906CEFE0F529A3E0F52AE52A453D
:103B5F002970099080027410F07F0022906FFCE0B2
:103B6F00FFF46030906CF1E06F6003023C02906FE5
:103B7F00FDE0FF906CF2E06F7079906FFEE0FF90C8
:103B8F006CF3E06F706D906FFFE0FF906CF4E06F7F
:103B9F006031805F906CF1E0906FFCF0906CF2E020
:103BAF00906FFDF0906CF3E0906FFEF0906CF4E08E
:103BBF00906FFFF0906CF5E0FFA3E0906CC3CFF037
:103BCF00A3EFF0906CEFE0702AA3E024F8F528E55E
:103BDF0031540744F0F58385328274082582F582CB
:103BEF00E43583F58363A201906CEF63A201AF28E4
:103BFF00123701AE29E4FCFDE532252AF532E53115
:103C0F003EF531ED3530F530EC352FF52FAF2EAECB
:103C1F002DAD2CAC2BAB32AA31A930A82FD3122B40
:103C2F00EC40099080027410F07F002290802CE508
:103C3F002FF0A3E530F0A3E531F0A3E532F090804B
:063C4F00027440F0AF28F2
:013C5500224C
:103C56009081E3E0F528052805280528052805288C
:103C66000528052805280528052890801CE0F52B41
:103C7600A3E0F52CA3E0F52DA3E0F52E9081E4E07A
:103C8600F5280528052805280528052805280528D6
:103C9600052805280528908020E0F52FA3E0F530BB
:103CA600A3E0F531A3E0F532E4F528E531B52D0AB8
:103CB600E532B52E05C21D023DACE531540744E898
:103CC600F58385328263A20190697E63A2017F0E2D
:103CD60012371790697EE0F529A3E0F52A906986E8
:103CE600E0FFF4604A906FF5E0FEEF6E7079A3E0B6
:103CF600FF906987E06F706F906FF7E0FF906988BB
:103D0600E06F7063906FF8E0FF906989E06F70571D
:103D1600906FF9E0FF90698AE06F704B906FFAE060
:103D2600FF90698BE06F703FE490698DF08008909A
:103D3600698D74FFF0D2D990697EE0702AA3E024E1
:103D4600F2F528E531540744E8F583853282740E8E
:103D56002582F582E43583F58363A20190697E634B
:103D6600A201AF28123717AE29E4FCFDE532252A59
:103D7600F532E5313EF531ED3530F530EC352FF5E0
:103D86002FAF2EAE2DAD2CAC2BAB32AA31A930A85D
:103D96002FD3122BEC5006E52A4529700990800195
:103DA6007410F07F0022908020E52FF0A3E530F01C
:103DB600A3E531F0A3E532F09080017440F0AF281E
:013DC60022DA
:0448B4008E318F3280
:1048B800908000E030E507906EF27401F02290726B
:1048C80039E0FCA3E0FDA3E0FEA3E0F5388E378DC8
:1048D800368C35E538FFE5375407FEE42FF534EE1E
:1048E80034C0F533853482F5837423F00534E53418
:1048F800700205335333C7F582853383740AF00594
:1049080034E534700205335333C7906CB863A201A1
:1049180085338385348263A2017F061236BB740611
:104928002534F534E43533F53385318385328263B4
:10493800A20185338385348263A20112369FE4FC89
:10494800FDFE907239E0F8A3E0F9A3E0FAA3E02FA6
:10495800FFEE3AFEED39FDEC38FCEF2408FFE43EAB
:10496800FEE43DFDE43CFC907239122C1D90723936
:10497800E0908040F090723AE0908041F090723B75
:10498800E0908042F090723CE0908043F09080008C
:034998007420F098
:01499B0022F9
:0A43DE008E2E8F2F8C308D318B3224
:1043E800908000E030E507906EF27401F022907240
:1043F80039E0FCA3E0FDA3E0FEA3E0F5388E378D9D
:10440800368C35E538FFE5375407FEE42FF534EEF2
:1044180034C0F533853482F5837423F00534E534EC
:10442800700205335333C7F582853383740AF00568
:1044380034E534700205335333C7906CB863A20176
:1044480085338385348263A2017F061236BB7406E6
:104458002534F534E43533F533852E83852F82638F
:10446800A20185338385348263A20112369F8F3976
:10447800EF2534F534E43533F533E532601785300C
:104488008385318263A20185338385348263A201E7
:10449800AF321236BBE53924082532F532FFE4FC89
:1044A800FDFEE5382FF538EE3537F537ED3536F5BD
:1044B80036EC3535F535908040E535F0A3E536F036
:1044C800A3E537F0A3E538F09080007420F0AF380A
:0C44D800AE37AD36AC35907239122C1D99
:0144E40022B5
:0250CC008F4112
:1050CE00908000E030E507906EF27401F02290724D
:1050DE0039E0FCA3E0FDA3E0FEA3E0F5458E448D90
:1050EE00438C42E545FFE5445407FEE42FFFEE34C2
:1050FE00C0906C2E63A201F5838F8263A201AF4133
:10510E001236BBE4FCFDFEE5452541F545EE354482
:10511E00F544ED3543F543EC3542F542908040E5DC
:10512E0042F0A3E543F0A3E544F0A3E545F09080FB
:10513E00007420F0AF45AE44AD43AC4290723912CC
:02514E002C1D16
:01515000223C
:06499C008E2B8F2CAB05F1
:1049A200908000E030E507906EF27401F022907280
:1049B20039E0FCA3E0FDA3E0FEA3E0F5328E318DE9
:1049C200308C2FE532FFE5315407FEE42FF52EEE51
:1049D20034C0F52D852E82F5837423F0052EE52E45
:1049E2007002052D532DC7F582852D83EBF0052E20
:1049F200E52E7002052D906CB863A201852D83858A
:104A02002E8263A2017F061236BB7406252EF52E76
:104A1200E4352DF52D532DC7E52B852E82852D836B
:104A2200F0052EE52E7002052D532DC7F582852D3A
:104A320083E52CF0052EE52E7002052D532DC7E5DA
:104A420032240AF532E43531F531E43530F530E41B
:104A5200352FF52F908040E52FF0A3E530F0A3E548
:104A620031F0A3E532F09080007420F0AF32AE3125
:0A4A7200AD30AC2F907239122C1DEC
:014A7C002217
:1053CB00908009E04480F09080E97441F07F09906F
:1053DB0080F6EFF0A37464F09080037402F0908079
:1053EB0003E020E1F9907135122C290000000090A8
:1053FB007135E0908064F0907136E0908065F090AC
:10540B007137E0908066F0907138E0908067F0A380
:10541B00E4F0A3F0A3F0A3F090803CF0A3F0A3F092
:02542B00A3F0EC
:01542D00225C
:1045E9009081E9E0F52E052E052E052E052E052EC6
:1045F900052E052E052E052E052E908034E0F52F6B
:10460900A3E0F530A3E0F531A3E0F5329081EAE0CB
:10461900F52E052E052E052E052E052E052E052E09
:10462900052E052E052E908038E0F533A3E0F534EC
:10463900A3E0F535A3E0F536E535B53108E536B53E
:1046490032037F0022E4F52EE535540744F8F5835B
:1046590085368263A20190713963A2017F06123700
:104669002F907139E064686014908038E52FF0A3C9
:10467900E530F0A3E531F0A3E532F0804C90713AD2
:10468900E02402F52EE535540744E0F583853682AA
:1046990063A20190713963A201AF2E12372FE4FC96
:1046A900FDFEE536252EF536EE3535F535ED353495
:1046B900F534EC3533F533908038E533F0A3E53440
:1046C900F0A3E535F0A3E536F09080037440F0AF30
:0146D9002EB2
:0146DA0022BD
:0246DB008F2E20
:1046DD009080E8E0640660037FFF22907135E0FC76
:1046ED00A3E0FDA3E0FEA3E0F5328E318D308C2FDB
:1046FD00E4FFFEFDFCAB32AA31A930A82FC3122B6B
:10470D00EC70609081F9E0F52F907135E0FCA3E03D
:10471D00FDA3E0FEA3E0FFE4FAF9F8EF2401FFEAC0
:10472D003EFEE93DFDE83CFC907135122C1D90716B
:10473D0035E0FCA3E0FDA3E0FEA3E0FFE4F8EF24E9
:10474D0001FFEA3EFEE93DFDE83CFC907135122C7F
:10475D001D908064E0F52FA3E0F530A3E0F531A3C3
:10476D00E0F53290713963A201E531540744D8F573
:10477D008385328263A201AF2E1236E9E4FCFDFE81
:10478D00E532252EF532EE3531F531ED3530F5309A
:10479D00EC352FF52F908064E52FF0A3E530F0A3D5
:1047AD00E531F0A3E532F09080037420F0AF32AE26
:0D47BD0031AD30AC2F907135122C1D7F00F6
:0147CA0022CC
:1058B900A2AF9224C2AF438E2075D2028F828E830B
:0C58C900E0FFE4F5D2538EDFA22492AF82
:0158D50022B0
:10584D00E5D220E0FBA2AF9224C2AF43D2028F82F9
:10585D008E83EDF075D25063D250A22492AFE5D273
:03586D0020E0FB3D
:015870002215
:10525900E4FDED2401FFE433FE1258B974B02DF5D5
:1052690082E4346CF583EFF00DBD3FE6E4FDED24F7
:105279007FFFE433FE1258B974A72DF582E4346A2E
:10528900F583EFF074A72DF582E4346AF583E070B5
:105299001B74A72DF582E4346AF5837420F074A891
:1052A9002DF582E4346AF583E4F080040DBD80BEF7
:1052B900E4906B26F0FDEDFF7E001258B974272D9E
:0D52C900F582E4346BF583EFF00DBDFEE9D6
:0152D60022B5
:02573E008B2DB1
:10574000A2AF9224C2AF85A22E53A2FE8E838F8277
:1057500005A28C838D827409123745E52D53A2FE74
:1057600043A22012374753A2DF852EA2A22492AF74
:01577000FF39
:015771002215
:1058D600A2AF9224C2AF8C838D82EF12374543A2CA
:0C58E6002012374753A2DFA22492AFFF2C
:0158F2002293
:025871008F287E
:10587300A2AF9224C2AFE4F5838D8274061237453A
:10588300E52843A22012374753A2DFA22492AF7F19
:015893000113
:0158940022F1
:025895008F285A
:10589700A2AF9224C2AFE4F5838D82740A12374512
:1058A700E52843A22012374753A2DFA22492AF7FF5
:0158B70001EF
:0158B80022CD
:10356E00A907E7FFA805EF93C3966008403B74FCDC
:10357E002FFF80F00F08EF93C3966008402B74FB6B
:10358E002FFF80E00F08EF93C3966008401B74FA7C
:10359E002FFF80D00F08EF93D3966008400B74F97D
:1035AE002FFF80C01F1F1F1F1FEF54FEF80303F7CE
:1035BE00E893FC08E893FD08E893FE08E893FF22E1
:1035CE0009E993C39D6008402974FB29F980F1092C
:1035DE00E993C39E6008401A74FA29F980E209E95A
:1035EE0093D39F6008400B74F929F980D3191919E8
:1035FE001919E9C313C313FF22740093F8ECC3988F
:10360E004024701F740193F8EDC398401970147420
:0E361E000293F8EEC398400E7009740393F8FF
:10362C00EFC39840037F00227F0122EDF8E6F008FB
:10363C00A3DFFA22EDF8E0F608A3DFFA22E0A36399
:10364C00A201F0A363A201DFF475A2002263A20120
:10365C00F0A363A20122E0A363A201F0A363A20181
:10366C00E0A363A201F0A363A201E463A201F0A3AF
:10367C0063A201DFE175A20022E0A363A2016DFE4B
:10368C00936CFDEE058393FC158363A201DFEA7551
:10369C00A200227F00E493A363A201F00F600CA3AD
:1036AC00E583C2E3F58363A20180EA75A20022E000
:1036BC00A363A201F0A3E583C2E3F58363A201DF58
:1036CC00EE75A20022E0A363A201F0A3E583C2E49D
:1036DC00D2E3F58363A201DFEC75A20022E0A363C1
:1036EC00A201F0A3E58344F8C2E5F58363A201DFF0
:1036FC00EC75A20022E583C2E3F583E0A363A2018B
:10370C00F0A363A201DFEE75A20022E583C2E4D22E
:0A371C00E3F583E0A363A201F0A32C
:1037260063A201DFEC75A20022E58344F8F583E08D
:10373600A363A201F0A363A201DFEE75A20022F942
:1037460022C002C004C00612FFF0D006D004D00288
:013756002250
:104D7C004572724C656E210A000A496E49503A0020
:104D8C00205544502054696D654750530A00200A41
:104D9C00495054696D653A2000200A4441544147FA
:104DAC0052414D3A20002049676E6F72650A20000F
:104DBC002043414E2054696D654750530A002054DE
:104DCC007261737353656E644552520A000ACEF8D1
:104DDC00C4EBE8EDFB43414E210A000A45727241D7
:104DEC00647243414E3A00205265496E6974204307
:104DFC00414E0A002043414E283029203E20544F7A
:104E0C00210A0020545520300A0020545520310A24
:014E1C000095
:03001E00E4FF22DA
:1057FE00C2A9438902758C48758A4875D90475DB30
:10580E004875DC4875DD4875DE48E4F5E9F5F9D2F2
:08581E00D9C2DAD28CD2DE22DD
:1057A500C2D990701BE07013E5E92419F5EB30D7E9
:1057B50006E5F904F5FB2285F9FB22E5E924C8F5A0
:0E57C500EB30D706E5F904F5FB2285F9FB224F
:10564B00C2D990701BE0702C303116E5E92432F58D
:10565B00EB30D707E5F904F5FB800385F9FBC23185
:10566B0022E5E92405F5EB30D706E5F904F5FB2235
:10567B0085F9FB22E5E92432F5EB30D706E5F90491
:07568B00F5FB2285F9FB226B
:105826001257FE90701BE0C3946450061251D512B5
:1058360057A5120022D230E4F557907133F0F546A1
:07584600F55BC231F55922A8
:10569200EF24FCF546D3940D4010201F077E4D7F6A
:1056A2007C1248B4E4F546D22E22906CF363A20138
:1056B20090712363A201AF46123649C22E201F0DFC
:0E56C2007E4D7F857C6C7DF3AB461243DE226D
:0F591D00D3EF6480948D5006E55B70028F5B22A0
:1023530020D903022489203003022489E55B70031A
:102363000223FC90697E540FFF7D48123640E548F6
:102373006401706990698DE0B4FF0ED232201F12A0
:102383007E4D7F8C1248B48009303206E4F55B023F
:1023930024891257A512542E854D11854E10854F51
:1023A3000F85500E124078E552F562E551F563AFA3
:1023B300097E007C037DE8122A93EF2563F563EE23
:1023C3003562F562850C6B201F0D7E4D7F9A7C690B
:1023D3007D7EAB5B1243DEE4F55B0224891257A5D5
:1023E30012542E201F0D7E4D7FA57C697D7EAB5B35
:1023F3001243DEE4F55B022489E5466055907127BC
:10240300E02405F528D3940D4007E4F546D22E8049
:1024130075907123E528540FFF7D48123640E54837
:1024230030E702D231E5486401701A303217E54BC8
:10243300B40112201F127E4D7FB27C697D7EAB5B9F
:102443001243DE800312542E1257A5E4F546D22E12
:102453008034E558601E907007540FFF7D48123694
:1024630040E548B4010320320312542E1257A5E469
:10247300F558801220010C90701BE0C39464500344
:10248300124A7D1257A5123DC78F28EF700302250C
:10249300E2E4F559E54830E70AE54BB41905D2D92A
:1024A3000225E212564BE5486401703BD232201FED
:1024B300077E4D7FBC1248B4854D11854E10854F64
:1024C3000F85500E124078E552F562E551F563AF82
:1024D300097E007C037DE8122A93EF2563F563EE02
:1024E3003562F562850C6BE55AC394C8501B3017EF
:1024F30018741C255AF582E43470F583E528255AAF
:10250300F55A7D48AF28123637301521E54820E7C4
:102513001C906EF37D48AF28123637AF28124C1C3F
:10252300EF700A201F077E4D7FCA1248B4E5485456
:102533008160030225E2E528D3940D4010301F0388
:102543000225E27E4D7FD91248B40225E2E54AD343
:102553009407401F301F030225E2906A7F7D48AF36
:10256300281236377E4D7FE77C6A7D7FAB28124386
:10257300DE806CE51230E66290725EE0FF9054BF3D
:1025830093FE547F65487052EFA393654A704B9056
:10259300725EE0C313FF2445F582E43472F583E0F1
:1025A300703853123F90725EE0FD744F2512F5822E
:1025B300E43462F583EEF0ED9054C093FE7450253D
:1025C30012F582E43462F583EEF074452FF582E46C
:1025D3003472F5837401F0431240AF2812309A30FD
:1025E30022269066DDE0C394FA5003E004F0301431
:1025F3001590701BE0C39464500C0559E55994F091
:102603004004C2AF80FEC222201603022731740A9F
:102613002563F563E43562F562FEAF63E4FCFD7B9D
:10262300607AEAF9F8D3122BD65011E4F562F56318
:10263300056BE56BC3943C4003E4F56BE5576031F0
:10264300D39401400415578028907133E004F0E0DF
:10265300D39403400D201F077E4D7FF31248B4121D
:102663005826201F077E4E7F001248B4E4F557D248
:1026730030302F43E558703F90700704F0A374087F
:10268300F0A37480F0A37401F0A37406F090711E9C
:10269300E090700CF090711FE090700DF09071203D
:1026A300E090700EF0907121E090700FF0E4A3F0D1
:1026B300A3F075580BC22F302D7290711CE070354A
:1026C300E55870319070077442F0A37408F090716C
:1026D3001DE0907009F0907122E090700AF0A374ED
:1026E30001F0755806201F077E4E7F0F1248B490E5
:1026F300711CE004F090711CE06402702FE55870C7
:102703002B9070077402F0A37408F090711DE09091
:102713007009F0A3F0A37401F0755806201F077E1B
:102723004E7F161248B490711CE004F0C216121AC0
:032733001AC214B3
:012736002280
:10577200E55A602CE4906DEFF0A3E55AF0906FF4D7
:10578200E0906DF1F0A37419F090701C63A2019087
:105792006DF363A201AF5A123649E4F55A7F012232
:0357A2007F002263
:0B592C00302E05C22E7F01227F0022DA
:0100210022BC
:06595100E4F55AF54622C0
:0A593700E4906A7FF0A3F0A3F022D1
:105490002043616E457247495400200A00457272EC
:1054A0004C656E43616E21000A002043616E4572B7
:1054B00072434821000A205265714572722100C46E
:1054C00000C401C402C403C404C405C406C407C89C
:1054D00000C801C802C803C804C805C806C807C276
:1054E00000C201C202C203C204C205C206C2070052
:0154F00000BB
:103DC700E59B541F6020201F1A7E547F901248B431
:103DD700E59B541FFF7E007D0312499C7E547F9A0A
:103DE7001248B4E4F59BE5BA30E010E4F5B375B1D9
:103DF70080F5B2D230F557907133F0E5CFF4700308
:103E0700023F1F752A01E4F529E5CFF4552A70030F
:103E1700023F0DE529C454F0F5B1E5B2547F6420A3
:103E27006003023EDEE5B3540FF54C85BC48E5BDA3
:103E3700541FFF131313541FFFE5BD54E044184FDD
:103E4700F549E5BDC43354E0FFE5BE131313541F12
:103E57004FF54AE5BEC43354E0FFE5BF13131354CF
:103E67001F4FF54B85A34D85A34E85A34F85A350C3
:103E770085A35185A35285A35385A354E4F5B220A6
:103E8700010FE548547EB5480843BDF875B3508027
:103E97000375B3D0E54C700AE548547EB548037FF7
:103EA7000022300108E54830E7037F0022E54CD3C4
:103EB7009408401D201F177E547F9D1248B4AF4CB5
:103EC7007E007D0312499C7E547FA81248B47F0070
:103ED70022E54C2405FF22E5B2549F6023201F20D2
:103EE7007E547FAA1248B4AFB27E007D0312499C6C
:103EF700AFB37E007D0312499C7E547FA81248B45D
:103F0700E4F5B275B3D0E52A25E0F52A0529E529B8
:0A3F1700C394085003023E107F001F
:013F2100227D
:10542E0090701BE0C39464505675B180E4F5B3F5EB
:10543E00B28548BCE54AC4135407FFE54954E04F12
:10544E00F5BDE54A33333354F8FFE54BC413540727
:10545E004FF5BEE54B33333354F8F5BF854DA38579
:10546E004EA3854FA38550A38551A38552A3855383
:10547E00A38554A3E54C540F2450F5B375570AC2B7
:02548E003022CA
:104A7D0075B190E5B220E613201F107E547FB5125C
:104A8D0048B4AFB27E007D0312499CE4F5B3F5B294
:104A9D00E51230E615E4F51290725EE02402F0E0C6
:104AAD009054BF93700490725EF0744F2512F5828E
:104ABD00E43462F583E0702D90725EE0FFC3132441
:104ACD0045F582E43472F583E0700543128080155C
:104ADD00E4F51290725EE02402F0E09054BF937002
:104AED000490725EF0E51230E72190725EE0FF9067
:104AFD0054BF93F5BCE4F5BDEFA393FF33333354AB
:104B0D00F8F5BE75BF784312408036744F2512F507
:104B1D0082E43462F583E0F5BC75BD8074502512D6
:104B2D00F582E43462F583E0FF33333354F8F5BE98
:104B3D0075BF7805120512E512C394324003E4F5F2
:054B4D001275B35022B7
:09594100EF6003C29622D2962207
:1051D50043AB01C2E8C2EAE4FFEFC454F0F5B1C342
:1051E500EF64809488500575B3D08003E4F5B3E48B
:1051F500F5B2F5BCF5BDF5BEF5BFF5C4F5C5F5C60B
:10520500F5C7F5A3F5A3F5A3F5A3F5A3F5A3F5A3B5
:10521500F5A30FBF0EC390701BE0FE25E0F5B47536
:10522500B50C75B66C75A11275AB0275C13E75C32B
:10523500FF75C203E490725EF0751280FF7F1990CE
:105245007245E4F0A3DFFCE4FF7F3290624FE4F0A7
:03525500A3DFFCD8
:015258002233
:103757000000000000000000000000000000000062
:103767003FF3630041D5E80043B71B8045984F00FE
:1037770047798280495C07804B3D3B004D1E6E8038
:103787004EFFA20050E2270052C35A8054A48E0075
:103797005685C180586846805A497A005C2AAD80B0
:1037A7005E0BE1005FEE660061CF998063B0CD00EC
:1037B70065920080677485806955B9006B36EC8027
:1037C7006D1820006EFAA50070DBD880000000009D
:1037D7000028DE80004DC8800076A700009E3400D8
:1037E70000C7123000EE9F8001177E0001405C8009
:1037F7000167E9800190C80001B8550001E13380F5
:10380700000000000028DE80004F1A000077F880D3
:10381700009F858000C8640000EFF1000118CF8089
:103827000141AE0001693B000192198001B9A680F0
:1038370001E2850000000000000151800002A300A2
:103847000003F48000054600000697800007E900A2
:1038570000093A80000A8C00000BDD80000D2F0064
:10386700000E8080000FD200001123800012750027
:103877000013C68000151800001669800017BB00EA
:1038870000190C80001A5E00001BAF80001D0100AC
:10389700001E5280001FA4000020F5800022470070
:1038A700002398800024EA0000263B8000278D0033
:1038B7000028DE800000000000000E1000001C2021
:1038C70000002A30000038400000465000005460D5
:1038D700000062700000708000007E9000008CA0E5
:1038E70000009AB00000A8C00000B6D00000C4E0F5
:1038F7000000D2F00000E1000000EF100000FD2002
:1039070000010B300001194000012750000135600C
:1039170000014370000151801F1C1F1E1F1E1F1F27
:043927001E1F1E1F22
:1041AD00E50825E025E02457F582E43437F5831240
:1041BD002BFD8F118E108D0F8C0EE508540370287A
:1041CD00E50D25E025E02403F582E43438F583126E
:1041DD002BFDEF2511F511EE3510F510ED350FF521
:1041ED000FEC350EF50E8026E50D25E025E024CFEC
:1041FD00F582E43437F583122BFDEF2511F511EE21
:10420D003510F510ED350FF50FEC350EF50EE50A01
:10421D0025E025E02437F582E43438F583122BFDB3
:10422D00EF2511F511EE3510F510ED350FF50FECFD
:10423D00350EF50EE50BC3940C402AE51124C0F59F
:10424D0011E51034A8F510E4350FF50FE4350EF532
:10425D000EE50B24F4FF7E007C0E7D10122A93AA2E
:10426D0006AB07800FAF0B7E007C0E7D10122A93DC
:10427D00AA06AB07AE02E4FCFDE5112BF511E51026
:10428D003EF510ED350FF50FEC350EF50EE50C7511
:10429D00F03CA4FFAEF0E4E5112FF511E5103EF56D
:1042AD0010ED350FF50FEC350EF50EE4FEE511258D
:1042BD0009F511EE3510F510ED350FF50FEC350E46
:0242CD00F50EEC
:0142CF0022CC
:10407800907261E0F50825E025E02457F582E434E4
:1040880037F583E508D3941F501DAF11AE10AD0F5F
:10409800AC0E123607EF700F74042582F582E435F2
:1040A80083F583050880DC74FC2582F58274FF356E
:1040B80083F583AF82122C0DC3E5119BF511E51032
:1040C8009AF510E50F99F50FE50E98F50E1508E528
:1040D8000814907261F0E508540370059038078061
:1040E800039037D3750D307F0D7D0E12356EA80401
:1040F800A905AA06C3E5119FF511E5109AF510E583
:104108000F99F50FE50E98F50E050D90383BAF1198
:10411800AE10AD0FAC0E7B007A00797C1235CE8FD5
:104128000AEF25E025E0243BF582E43438F58312D4
:104138002C0DC3E5119BF511E5109AF510E50F99C3
:10414800F50FE50E98F50E050A9038BBAF11AE10C5
:10415800AD0FAC0E7B007A00795C1235CE8F0BEF79
:1041680025E025E024BBF582E43438F583122C0DD4
:10417800C3E5119BF511E5109AF510E50F99F50FB8
:10418800E50E98F50EAE10AF117C007D3C122AA505
:104198008D09AE10AF117C007D3C122AA58E108FC0
:0541A8001185110C223D
:101EBD003E2A2C312CCFE0F0E0ECE5F2F0FB20F3E4
:101ECD00EFF0E0E2EBFFFEF9E5E3EE20EAEEEDF2F6
:101EDD00F0EEEBEBE5F0E020CACF20C8F1E5F2FC27
:101EED000A003E4C2C6B30312C25732C43EAEEF05E
:101EFD00EEF1F2FC20EDE020F8E8EDE52043414E57
:101F0D002C30202D20353030EAE1283530EC292CCD
:101F1D0031202D203530EAE128353030EC290A000A
:101F2D0030202D20353030EAE1283530EC290031D4
:101F3D00202D203530EAE128353030EC29003E42A5
:101F4D002C6330312C2562752CC2F2EEF0E8F7EDE2
:101F5D00FBE920EAEEEDF2F0EEEBEBE5F020EDE043
:101F6D0020F8E8EDE50A003E2A2C312CCFE0F0E018
:101F7D00ECE5F2F0FB20EFF0EEF2EEEAEEEBE02016
:101F8D00CCDDCA203837302D352D31303428313065
:101F9D0031290A003E4C2C6B30352C256C752C28C4
:101FAD0031303129D1EAEEF0EEF1F2FC20EEE1EC28
:101FBD00E5EDE020EDE020EFEEF0F2F32C313030E6
:101FCD002C3230302C3330302C3630302C31323006
:101FDD00302C323430302C343830302C39363030DF
:101FED002C31393230302C33383430302C353736C3
:101FFD0030302C3131353230300A003E532C6B30BD
:10200D00362C2562752C2831303129CDEEECE5F0DA
:10201D0020F1F2E0EDF6E8E80A003E532C6B303784
:10202D002C2562752CC0E4F0E5F120415344550A8E
:10203D00003E532C6B30382C256C752CCDE0F7E021
:10204D00EBFCEDFBE920E0E4F0E5F120D2D10A0054
:10205D003E532C6B30392C256C752CCDE0F7E0EB15
:10206D00FCEDFBE920E0E4F0E5F120D2C8D20A0056
:10207D003E532C6B31302C256C752CCDE0F7E0EBFD
:10208D00FCEDFBE920E0E4F0E5F120D2C8C80A0040
:10209D003E532C6B31312C256C752CCDE0F7E0EBDC
:1020AD00FCEDFBE920E0E4F0E5F120D2D30A003E9F
:1020BD00532C6B31322C2562752CD0E0E7ECE5F01A
:1020CD0020C0D1C4D328312032290A003E532C6BB5
:1020DD0031332C2562752CD0E0E7ECE5F020EFF0E4
:1020ED00E8F7E8EDFB20EFE5F0E5E4E0F7E828316F
:1020FD002032290A003E532C6B31342C2562752C6D
:10210D00D0E0E7ECE5F020E0E4F0E5F1E020EEE1F1
:10211D00FCE5EAF2E028322033290A003E422C6B1E
:10212D0031362C2562752CCFE5F0E5E4E0F7E020A3
:10213D00D2C8D220F120E2F0E5ECE5EDE5EC0A00A5
:10214D003E532C6B31372C2562752C2831303429B8
:10215D00CAEEEB20EFE0EAE5F2EEE220EDE020EA58
:10216D00E2E8F20A003C21003C6B30313D003C635B
:10217D0030313D003C6B30353D003C6B30363D0021
:10218D003C6B30373D003C6B30383D003C6B30399B
:10219D003D003C6B31303D003C6B31313D003C6BC3
:1021AD0031323D003C6B31343D003C6B31333D00F1
:1021BD003C6B31353D003C6B31363D003C6B31376E
:1021CD003D000A414F75743A0043414E205455204D
:1021DD004F4B0A0043414E205455205265710A0061
:1021ED00496E69745443500A00436F6E6E65637493
:1021FD005443500A004C697374656E5443500A0081
:10220D00534F434B5F5443505F45535441424C49E8
:10221D00534845440A002054552054696D654F5567
:10222D0054210A000A2D3E20000A4173496E000A0E
:10223D003ED1E1F0EEF1CAE0EDE0EBE0203A3C28D2
:10224D00CAE2F229000A3ED1E1F0EEF1CFF0EEF64E
:10225D00E5E4F3F0203A3C28CAE2F229000A3E00F8
:10226D003A3C28CAE2F229000A3ED1F2E0F2F3F13B
:10227D00CAE0EDE0EBE03F203A3C28CAE2F229004B
:10228D000A3EC7E0EFF0EEF13A003C28CDE5F2C48E
:10229D00E0EDEDFBF529003E3F3F3F3A0020D2D364
:1022AD00200020C2FBE1EEF0200020C8F1EFEEEBA4
:1022BD00EDE8F2FC200020CEF2ECE5EDE020002070
:1022CD00C2F0E5ECFF200020CEEFF0EEF120002073
:1022DD00C7E0E2E5F0F8E5EDE8E5C8EDE8F6E8E0A1
:1022ED00EBE8E7E0F6E8E8200020CAE2E8F2D2D316
:1022FD00200020CEF8E8E1EAE0D2D3200020D2D3AE
:10230D0020C3EEF2EEE2EE200020D2D320C2FBEF8E
:10231D00EEEBEDE5EDEE200020D2D1F1200020C056
:10232D00EAF2E2F6CEEFF0EEF1E0200020D2D1F6A7
:10233D00200020D2C8D2F6200020D2C8C82000200C
:06234D00D2C8D2F120000D
:030023000242D0C6
:0B42D000C0E0C083C082C0D075D018D1
:1042DB0020980302439FC298757401AF993006036F
:1042EB000243D5D291200228BF680DD202D20E759F
:1042FB00640075680002439FEF6410600302439FE4
:10430B00D202D20F7570027568037564000243D533
:10431B00E56870078F7005680243D5E568B4010F37
:10432B00E570B51F0505680243D5C2020243D5E50A
:10433B0068B4020AEF646860CEC2020243D5E56836
:10434B00B4031E74382569F582E43467F583EFF006
:10435B0005692564F5641570E570706E75680480E9
:10436B0069E568B4040DE564B51F040568805BC29C
:10437B00028057E568B4051CBF160ED2068569701E
:10438B00756900C202C2918041C20FC20E756900ED
:10439B00C202803630993330032E90620DE0FFE578
:1043AB006CC39F4008C203D210C290801BD2907482
:1043BB0078256CF582E43468F583E0F56F526FA2D3
:0A43CB00D0929B856F99056CC29992
:0943D500D0D0D082D083D0E032B8
:103F22007BFF7A1E79BD12279990701BE070147581
:103F320030FF75311F75322D7BFF7A1E79EF122704
:103F42009980127530FF75311F75323C7BFF7A1EE6
:103F520079EF1227997BFF7A1F794BA201E433F59F
:103F6200301227997BFF7A1F79741227999069780A
:103F7200E0FEA3E0FFC3E49FFFE49EFEAB07FA333B
:103F820095E0F9F87F007E8C7D0A7C00122B368F3B
:103F9200338E328D318C307BFF7A1F79A1122799B3
:103FA2007BFF7A2079089064D2E0F5301227997B62
:103FB200FF7A207927906100E0F5301227997BFF84
:103FC2007A20793E9064D3E0FEA3E0FFE48F338E43
:103FD20032F531F5301227997BFF7A20795D9062B4
:103FE2000BE0FEA3E0FFE48F338E32F531F53012A1
:103FF20027997BFF7A20797D906209E0FEA3E0FF9A
:10400200E48F338E32F531F5301227997BFF7A2017
:10401200799D9066E8E0FEA3E0FFE48F338E32F5EF
:1040220031F5301227997BFF7A2079BCA205E4335F
:1040320004F5301227997BFF7A2079D9A204E43360
:1040420004F5301227997BFF7A217902A20BE4331F
:104052002402F5301227997BFF7A217929A212E4F2
:1040620033F5301227997BFF7A21794D906737E03B
:06407200F530122799222F
:10335C007E217F72125047EF4E70037F0122E49062
:10336C00701BF07E217F75125047EF4E601512587E
:10337C00F3BF310690701B740AF0BF320690701BBD
:10338C007464F07E217F7B125047EF4E600D125417
:10339C00F1EC4D4E4F24FF92018002C2017E217F41
:1033AC0081125047EF4E60231254F1A804A905AACC
:1033BC0006AB077F007E8C7D0A7C00122B36122B0D
:1033CC00C8906978EEF0A3EFF0800A90697874FDEC
:1033DC00F0A374C0F07E217F87125047EF4E600A35
:1033EC001254F19064D2EFF080069064D27401F024
:1033FC007E217F8D125047EF4E600A1254F190617E
:10340C0000EFF080089064D2E0906100F07E217FA4
:10341C0093125047EF4E600D1254F19064D3EEF0BE
:10342C00A3EFF080089064D3E4F0A304F07E217F36
:10343C0099125047EF4E600D1254F190620BEEF062
:10344C00A3EFF0800A90620B7403F0A374E9F07E92
:10345C00217F9F125047EF4E600D1254F19062097C
:10346C00EEF0A3EFF0800A906209740BF0A374B92C
:10347C00F07E217FA5125047EF4E600D1254F19053
:10348C0066E8EEF0A3EFF0800A9066E87407F0A30C
:10349C0074D1F07E217FAB125047EF4E601C12545A
:1034AC00F1EF24FFFFEE34FFFEED34FFFDEC34FFB3
:1034BC00FC4D4E4F24FF92058002C2057E217FB148
:1034CC00125047EF4E601C1254F1EF24FEFFEE3405
:1034DC00FFFEED34FFFDEC34FFFC4D4E4F24FF920C
:1034EC000B8002C20B7E217FB7125047EF4E601C3F
:1034FC001254F1EF24FFFFEE34FFFEED34FFFDEC30
:10350C0034FFFC4D4E4F24FF92048002C2047E21F6
:10351C007FBD125047EF4E600D1254F1EC4D4E4FE3
:10352C0024FF92098002D2097E217FC3125047EFFB
:10353C004E600D1254F1EC4D4E4F24FF921280024E
:10354C00D2127E217FC9125047EF4E600A1254F1FD
:10355C00906737EFF080069067377401F0C20A7FEE
:01356C00005E
:01356D00223B
:1047CB00E4F56C74DE256CF582E43466F583E4F075
:1047DB0074D5256CF582E43466F583E4F074C92551
:1047EB006CF582E43463F583E4F0056CE56CB40896
:1047FB00D2E4F56C7438256CF582E43468F583E407
:10480B00F0056CE56CB440ECE4F56C7481256CF54B
:10481B0082E43462F583E4F0056CE56CB480ECE47F
:10482B00F56EF56D907261F0C203C2089066E7F009
:10483B00C211C207C210C202C206F56C90620DF023
:10484B00F560F569F574C200C213C20D90697874F6
:10485B00FFF0A374F4F07565FF9061017402F0A38F
:10486B00F090624EF012335CE4F512C291C290C22A
:10487B00ADF5C9D2CDD2CCC2C9C2CAF5CDF5CC905B
:10488B006978E0F5CBA3E0F5CA85CBCD85CACCD250
:10489B009FD29ED29CD2CAC2ACC298C29975B81094
:0948AB0075B710D2AC1253CB22F8
:024CCC008F2E29
:104CCE00E4FF7C617D03FEEEC3952E50120DEDAA1E
:104CDE000470010C14F5828A83E02FFF0E80E80D1C
:104CEE00EDAA0470010C14F5828A83EFF00DEDAE7F
:104CFE000470010C14F5828E837416F0052E052EA9
:104D0E007E687F787C617D03E52EB4040E8F828EE3
:104D1E00837410F00FBF00010E80328F828E837469
:104D2E0068F00FBF00010EE52E24FEFB8F828E83EE
:104D3E00F00FBF00010E8F828E83EBF00FBF0001CC
:104D4E000E8F828E837468F00FBF00010E8C838DE0
:104D5E008263A2018E838F8263A201AF2E12364927
:0D4D6E00E52EB4040304FF22E52E2404FF0B
:014D7B002215
:10570800200332124CCC90620DEFF030210D7E2137
:105718007FCF7C687D78E0FB1243DE300D057F018A
:10572800125941E5606003F57122E49066DDF0F5F9
:065738006CD203D299229D
:02309A008F297C
:10309C00E54824BE700302332824FA70030232225E
:1030AC002404600302335BE54930E70302314BE54E
:1030BC004B6066E54AC39402400302335BE54A70F9
:1030CC0007E54B14F52A8006E54B241FF52AE52A63
:1030DC0075F004A424D2F582746335F0F5837D4D2C
:1030EC007F04123637E52A75F004A424C9F58274DE
:1030FC006235F0F5837D517F0412363774C1254A51
:10310C00F582E43462F5837481F07481252AF582AA
:10311C00E43462F5837401F02274D5254AF582E417
:10312C003466F583E04481F0E54A25E025E0240B84
:10313C00F582E43467F5837D4D7F0412363722E542
:10314C004C6408600302335B752901E54B5407FF9F
:10315C00E529A807088002C333D8FCF52974082593
:10316C006EF56EB56D067408256DF56DE54B547FE7
:10317C00FFE54AC43354E02FFE7400256EF582E45B
:10318C003460F583EEF0E54BC39480503CEF1313A1
:10319C0013541FFFE54A25E025E025E025E0240B2C
:1031AC00F582E43467F583E5822FF582E43583F507
:1031BC0083E0FFE529F4FEEF5EF07401256EF582E5
:1031CC00E43460F583E4F0803AE54B547FFF13134D
:1031DC0013541FFFE54A25E025E025E025E0240BEC
:1031EC00F582E43467F583E5822FF582E43583F5C7
:1031FC0083E04529F07401256EF582E43460F58393
:10320C007401F07402256EF582E43460F5837D4D13
:10321C007F0612363722E54B54E06440702CE54BA8
:10322C00540F144440FF74C9254AF582E43463F505
:10323C0083EFF0E54A25E025E024EAF582E43466E4
:10324C00F5837D4D7F041236372274C9254AF582E9
:10325C00E43463F583E0F50CE54B547FFF13135412
:10326C003FF50AE54A75F008A4250AF50DE50C3082
:10327C00E657540FB50A2D301216E50C540744903E
:10328C00FE74C9254AF582E43463F583EEF08014AC
:10329C00E50C54074410FE74C9254AF582E43463E6
:1032AC00F583EEF03012117438250DF582E4346894
:1032BC00F583E054FEF080207438250DF582E4345B
:1032CC0068F583E04403F0800F7438250DF582E433
:1032DC003468F583E04403F075F040E54AA424D546
:1032EC00F582E5F03464F58375F002EF122C5A7D0B
:1032FC004DAF4C123637303256740E250DF582E434
:10330C003462F583E56BF0E50D25E02486F582E467
:10331C003461F583E562F0A3E563F022302D30E5EE
:10332C004BB40112201F077E217FD61248B4E54E04
:10333C0004907134F022E54BB4031490711CE0B48A
:0F334C0001037405F0201F077E217FE11248B4B2
:01335B00224F
:101A1A00201403021B119080E8E0700F1253CB30A0
:101A2A0021077E217FED1248B4C20C9080E8E06461
:101A3A000E6003021ADA200A03021AC59080F0F037
:101A4A00906185E0FF04F0EF30E025906CC7E0FF7D
:101A5A0060419080F0F0906CC8E09080F1F0906C5A
:101A6A00C9E09080F2F0906CCAE09080F3F0802395
:101A7A00906CCBE0FF601C9080F0F0906CCCE09012
:101A8A0080F1F0906CCDE09080F2F0906CCEE09016
:101A9A0080F3F07529099080F4E529F0752964A38B
:101AAA00E529F09080F0E060229080037404F03021
:101ABA0021197E217FF61248B480109080037408A1
:101ACA00F03021077E227F021248B4C20C7561559C
:101ADA009080E8E0B4060D200C0A3021077E227FB0
:101AEA000D1248B4E56A6002156AC214302D1890C6
:101AFA006206E004F0E0D39414400C201F077E2213
:101B0A007F231248B4C22D9066E7E0704B90670AB3
:101B1A00E004F0E0FFD394074007E56160037561D4
:101B2A0003EF540790670AF0E0FF24C9F582E43412
:101B3A0063F583E0FE30E72074C92FF582E434634D
:101B4A00F583EE547FF074C92FF582E43463F5838C
:101B5A00E0540F049066E7F020112A906207E0042F
:101B6A00F0E0543FF0E0FF2438F582E43468F5836E
:101B7A00E0FE30E010D21174382FF582E43468F5B3
:101B8A0083EE54FEF02007269066E6E004F0E05467
:101B9A003FF0E0FF2481F582E43462F583E0600ED1
:101BAA00D20774812FF582E43462F583E4F02008C9
:101BBA002A906208E004F0E05407F0E0FF24D5F52B
:101BCA0082E43466F583E0FE30E71074D52FF5829F
:101BDA00E43466F583EE547FF0D208300C63E56A8C
:101BEA00705F7E717F3F1208858F29E529605290C8
:101BFA00713BE55FF0E55EA3F0A3E55DF0E55CA36C
:101C0A00F03005020529300B0205293004020529A6
:101C1A00E529240490713AF0E5292406FF1246DBEF
:101C2A007402255FF55FE4355EF55E9063D1E004EA
:101C3A00F0906737E0FF9063D1E0C39F4003756A75
:101C4A00041245E98F29E5297003021D0030210C91
:101C5A007E227F317C717D39FB1243DE90713BE03D
:101C6A00B4071C740BF07F061246DBE4F55EF55FE1
:101C7A00F55CF55DD20CF56A9063D1F0756155900B
:101C8A00713BE0B443087483F07F061246DB90711F
:101C9A003BE0B4130A7423F07F061246DBC20C90B1
:101CAA00713BE0FFB40107E4F56A9063D1F0EF20DD
:101CBA00E04690713A7404F0A3E0752C00F52DA368
:101CCA00E0FEE4EE422C7402252DF52DE4352CF5C8
:101CDA002C90713B7401F0E4A3F0A3E52DF0E52C00
:101CEA00A3F07F061246DB852C5C852D5D7E717F15
:101CFA003F122DAD8002C21E200603021EBCE570F3
:101D0A0054802438F582E43467AF82F52A8F2B3069
:101D1A0021107E227F36E570547FFBAD2BAC2A1250
:101D2A0043DE200E06200F03021EBA852B82852A67
:101D3A0083A3E0FF9064D2E0FEEF6E6003021EB65A
:101D4A00E52B2407F582E4352AF583E0FEE52B240A
:101D5A0006F582E4352AF583E07C002400F52DECB3
:101D6A003EF52C852B82852A83E0544F24BF60469A
:101D7A0024FE6064147003021E1724FB7003021E03
:101D8A0030147003021E4F147003021E4F240B609E
:101D9A0003021EAC201F077E227F3C1248B4E49047
:101DAA006103F09064D2E0906104F07F0212570858
:101DBA00756155021EB6201F077E227F521248B453
:101DCA00E4906103F09064D2E0906104F07F021223
:101DDA005708756155021EB6201F077E227F6A12B8
:101DEA0048B4E4906103F09064D2E0906104F07F1B
:101DFA0002125708201F077E227F6D1248B4E52B76
:101E0A002402FFE4352AFE122DAD021EB6201F075A
:101E1A007E227F6A1248B4E52B2402FFE4352AFEAB
:101E2A00122DAD021EB6201F077E227F751248B4FE
:101E3A00906103740BF09064D2E0906104F07F0229
:101E4A001257088067201F077E227F8D1248B47EB2
:101E5A00617F051208858F29E5296027906103743F
:101E6A0008F09064D2E0906104F030050205293050
:101E7A000B0205293004020529E5292402FF12571D
:101E8A000880299061037409F09064D2E09061049B
:101E9A00F07F02125708201F137E227F971248B440
:101EAA00800A201F077E227FA41248B4C20FC20EE6
:021EBA00C2065E
:011EBC002203
:102DAD008E2E8F2F8F828E83E0249C7003022FE74F
:102DBD0024FD7003022F08243A6003023099201F6E
:102DCD00077E227FAA1248B4852E83852F8263A2A7
:102DDD000190672B63A2017F0B123649852F8285E7
:102DED002E83A3A3E0543FF50A7403252FF52FE49A
:102DFD00352EF52E300408052FE52F7002052E8592
:102E0D002F82852E83E0FF906100E0FEEF6E600360
:102E1D00023099052FE52F7002052E300508052F7C
:102E2D00E52F7002052E852F82852E83E0756600B5
:102E3D00F567052FE52F7002052EF582852E83E0AF
:102E4D00FEE4EE4266052FE52F7002052E9066E832
:102E5D00E0FEA3E0FFC3E5679FF567E5669EF566B7
:102E6D00D3E5679480E56694004003023099300BFA
:102E7D0008052FE52F7002052E852F82852E83E004
:102E8D00F50CE50A64067066E50C30E742201F0775
:102E9D007E227FAF1248B4302D03023099D22DE43B
:102EAD0090711CF0906206F0E566C4F854F0C868A5
:102EBD00E567C4540F4890711DF0E567540F25E088
:102ECD00FFE433E50C640154012F907122F02220B0
:102EDD001F077E227FB71248B4202D030230999030
:102EED00711CE0640660030230997402F022201F09
:102EFD00077E227FC31248B4C22D22201F077E22D7
:102F0D007FCC1248B47406252FF52FE4352EF52EFF
:102F1D00300508052FE52F7002052E300B08052F03
:102F2D00E52F7002052E300408052FE52F700205E0
:102F3D002E052FE52FAE2E7002052E14F5828E83F1
:102F4D00E0756600F567052FE52FAE2E7002052E94
:102F5D0014F5828E83E0FEE4EE4266052FE52FAE7A
:102F6D002E7002052E14F5828E83E0F50C052FE5EB
:102F7D002FAE2E7002052E14F5828E83E0F50B0513
:102F8D002FE52FAE2E7002052E14F5828E83E0F5FF
:102F9D000A052FE52FAE2E7002052E14F5828E83B5
:102FAD00E0F50D052FE52FAE2E7002052E14F582DE
:102FBD008E83E0F508AE66AF677C037DE8122AA527
:102FCD008F091241AD90711EE511F0A3E510F0A32C
:102FDD00E50FF0A3E50EF0D22F22201F077E227FF2
:102FED00D41248B4E5616003023099852F82852E95
:102FFD0083A3A3E0640660030230997406252FF5C0
:10300D002FE4352EF52E300508052FE52F7002051E
:10301D002E300B08052FE52F7002052E3004080504
:10302D002FE52F7002052E852F82852E83E06414E7
:10303D00705AE4F50C74D5250CF582E43466F583ED
:10304D00E030E00E74D5250CF582E43466F583741A
:10305D0083F074C9250CF582E43463F583E0FF3009
:10306D00E40F74C9250CF582E43463F583EF44A0B5
:10307D00F0050CE50CB408BD90620874FFF0906784
:0D308D000AF0E49066E7F0C20875610122C8
:1057D3008E318F32300404E4123659906100E012A6
:1057E3003659300504E4123659E532123659E5319B
:0B57F300123659300B04E41236592224
:040885008E2E8F2FF5
:10088900E56164557036201F077E227FDC1248B46B
:1008990063A201852E83852F8263A201E4F5617429
:1008A9004612365974011236597404123659E4FF46
:1008B900FE1257D374021236597F0722202D0302E4
:1008C9000992907134E0605190672B63A201852EE3
:1008D90083852F8263A2017F0B123649907134E020
:1008E900B40117201F077E227FF61248B4852F8294
:1008F900852E83A3A3740AF08015201F077E227F0B
:10090900FF1248B4852F82852E83A3A37447F0E490
:10091900907134F0C22D7F072290711CE06405703C
:1009290031201F077E237F0A1248B490672B63A2E8
:1009390001852E83852F8263A2017F09123649859D
:100949002F82852E83A3A37407F090711C14F07F66
:10095900072290711CE06403702F201F077E237FFC
:10096900161248B490672B63A201852E83852F82C6
:1009790063A2017F09123649852F82852E83A3A39D
:100989007407F090711CF0FF22E56E656D7003022B
:100999000A90201F077E237F251248B4E56D24089D
:1009A900F5307408256DF56DD21374022530F58282
:1009B900E43460F583E0F51174032530F582E434FD
:1009C90060F583E0F51074042530F582E43460F5B0
:1009D90083E0F50F74052530F582E43460F583E092
:1009E900F50E12407874072530F582E43460F583FA
:1009F900E0FE74062530F582E43460F583E0FDEE0F
:100A0900F566EDF567AF097E007C037DE8122A9350
:100A1900EF2567F567EE3566F56663A201852E83D6
:100A2900852F8263A201741E123659740112365938
:100A3900740312365974002530F582E43460F58365
:100A4900E0FF9064D4E02FFF9064D3E03400FE12FD
:100A590057D374012530F582E43460F583E012360A
:100A690059E567123659E566123659E50C123659B9
:100A7900E50B123659E50A123659E50D123659E5D4
:100A8900081236597F0E22E56130E045201F077EA6
:100A9900237F2B1248B463A201852E83852F82639D
:100AA900A20174641236597401123659E561B40110
:100AB9000A74071236597561028008740A12365988
:100AC900E4F561E4FFFE1257D374141236597F0717
:100AD90022200803020B90201F077E237F3912482A
:100AE900B4C20863A201852E83852F8263A2017493
:100AF9000112365974A0123659906208E024D5F5CE
:100B090082E43466F583E030E118741412365990A2
:100B19006208E024D5F582E43466F583E054FDF0FB
:100B290080057402123659906208E075F020A4FF1E
:100B39009064D4E02FFF9064D3E035F0FE1257D3D0
:100B4900E4F530906208E025E025E0240BF582E425
:100B59003467F583E5822530F582E43583F583E052
:100B6900F50AE4F50CE50A5401123659E50AC313EE
:100B7900F50A050CE50CC3940840EA0530E530C3D5
:100B8900940440BF7F26229066E7E07003020D0CB3
:100B9900201F077E237F3F1248B49066E7E025E0D7
:100BA90025E0F50CE4F063A201852E83852F82638D
:100BB900A20190670AE0FF24C9F582E43463F58352
:100BC900E0FE30E55B74C92FF582E43463F583EE0A
:100BD90054DFF07409123659E50C24801236597421
:100BE9001412365990670AE075F020A4FF90620C40
:100BF900E02FFF90620BE035F0FE1257D390670AA1
:100C0900E075F040A424D5F582E5F03464F583AFAE
:100C19000C123662E50C75F003A4F5302406FF22A8
:100C2900301213740A123659E50C2480123659749D
:100C39000312365980117409123659E50C248012B1
:100C49003659740112365990670AE075F020A4FFED
:100C590090620CE02FFF90620BE035F0FE1257D343
:100C690090670AE075F040A424D5F582E5F0346474
:100C7900F583AF0C123662E50C75F003A4F530303C
:100C8900127B252FF52FE4352EF52E90670AE0FF0C
:100C990025E025E024EAF582E43466F583E0F511E0
:100CA900EF25E025E024EBF582E43466F583E0F5F1
:100CB9001090670AE0FF25E025E024ECF582E43492
:100CC90066F583E0F50FEF25E025E024EDF582E4F4
:100CD9003466F583E0F50E124078AF097E007C0397
:100CE9007DE8122A938E668F67EF123659E56612F0
:100CF9003659E50C123659E5302409FF22E530242E
:100D090006FF22200703020E23201F077E237F46AA
:100D19001248B4C20763A201852E83852F8263A27C
:100D29000174251236597401123659740112365953
:100D39009066E6E0FF90620AE02FFF906209E034D6
:100D490000FE1257D39066E6E025E025E0F530FF76
:100D5900053074D22FF582E43463F583E0123659F5
:100D6900AF30053074D22FF582E43463F583E01295
:100D79003659AF30053074D22FF582E43463F583E8
:100D8900E0123659AF30053074D22FF582E434635E
:100D9900F583E0123659E412365974FC2530F530E2
:100DA900FF053074C92FF582E43462F583E0F5114B
:100DB900AF30053074C92FF582E43462F583E0F56C
:100DC90010AF30053074C92FF582E43462F583E041
:100DD900F50FAF30053074C92FF582E43462F5831D
:100DE900E0F50E124078AF097E007C037DE8122AF7
:100DF900938E668F67EF123659E566123659E50C00
:100E0900123659E50B123659E50A123659E50D1213
:100E19003659E5081236597F1222201103020EFABB
:100E2900201F077E237F4C1248B4C21163A201859B
:100E39002E83852F8263A201A23282125071740A15
:100E4900123659748412365974031236599062074E
:100E5900E075F004A4FF90620CE02FFF90620BE0B4
:100E690035F0FE1257D3906207E075F008A424D537
:100E7900F582E5F03464F5837F04123662906207E7
:100E8900E025E02486F582E43461F583E0F566A384
:100E9900E0F567123659E566123659906207E02483
:100EA9000EF582E43462F583E01236597F15227417
:100EB90009123659748412365974021236599062DD
:100EC90007E075F004A4FF90620CE02FFF90620B1D
:100ED900E035F0FE1257D3906207E075F008A424BC
:100EE900D5F582E5F03464F5837F041236627F120A
:030EF900227F0055
:010EFC0022D3
:0100220022BB
:104EB900020EFDE493A3F8E493A34003F68001F204
:104EC90008DFF48029E493A3F85407240CC8C333FA
:104ED900C4540F4420C8834004F456800146F6DFC9
:104EE900E4800B010204081020408090594AE47EB6
:104EF900019360BCA3FF543F30E509541FFEE493BE
:104F0900A360010ECF54C025E060A840B8E493A384
:104F1900FAE493A3F8E493A3C8C582C8CAC583CAAF
:104F2900F0A3C8C582C8CAC583CADFE9DEE780BE67
:015950000056
:102A9300EF8DF0A4A8F0CF8CF0A428CE8DF0A42E57
:022AA300FE2211
:102AA500BC000BBE0029EF8DF084FFADF022E4CC15
:102AB500F875F008EF2FFFEE33FEEC33FCEE9DECDE
:102AC500984005FCEE9DFE0FD5F0E9E4CEFD22ED24
:102AD500F8F5F0EE8420D21CFEADF075F008EF2F6E
:102AE500FFED33FD4007985006D5F0F222C398FD5F
:052AF5000FD5F0EA22FC
:102AFA0075F008758200EF2FFFEE33FECD33CDCC93
:102B0A0033CCC58233C5829BED9AEC99E582984015
:102B1A000CF582EE9BFEED9AFDEC99FC0FD5F0D6F2
:102B2A00E4CEFBE4CDFAE4CCF9A88222B800C1B91C
:102B3A000059BA002DEC8BF084CFCECDFCE5F0CB5A
:102B4A00F97818EF2FFFEE33FEED33FDEC33FCEB93
:102B5A0033FB10D703994004EB99FB0FD8E5E4F94E
:102B6A00FA227818EF2FFFEE33FEED33FDEC33FC3B
:102B7A00C933C910D7059BE99A4007EC9BFCE99A2F
:102B8A00F90FD8E0E4C9FAE4CCFB2275F010EF2F74
:102B9A00FFEE33FEED33FDCC33CCC833C810D70774
:102BAA009BEC9AE899400AED9BFDEC9AFCE899F8AF
:0E2BBA000FD5F0DAE4CDFBE4CCFAE4C8F92242
:0E2BC800C3E49FFFE49EFEE49DFDE49CFC221E
:102BD600EB9FF5F0EA9E42F0E99D42F0EC6480C876
:062BE60064809845F02216
:102BEC00EB9FF5F0EA9E42F0E99D42F0E89C45F03F
:012BFC0022B6
:102BFD00E493FC740193FD740293FE740393FF221E
:102C0D00E493F8740193F9740293FA740393FB221D
:0C2C1D00ECF0A3EDF0A3EEF0A3EFF0222A
:102C2900A8828583F0D083D082122C40122C4012C6
:102C39002C40122C40E473E493A3C583C5F0C583EB
:102C4900C8C582C8F0A3C583C5F0C583C8C582C8F5
:012C59002258
:0C2C5A00A42582F582E5F03583F5832285
:10273700E53C2430F8E6053C22782D302B02783032
:10274700E475F001122D0D022C662024EB7F2ED2AA
:10275700248018EF540F2490D43440D4FF30280B32
:10276700EF24BFB41A0050032461FFE53D60021552
:102777003D0540E5407002053F302B0D782DE4758F
:10278700F001122D0DEF022CAC0256047403D22B6C
:102797008003E4C22BF53C8B2D8A2E892FE4F53D6F
:1027A700F53FF540E53D60077F2012277280F575FC
:1027B7003EFFC225C224C226C227C229C22AC22C72
:1027C700122740FF700D302B057F00122783AF4083
:1027D700AE3F22B4255FC2D5C228122740FF24D0BE
:1027E700B40A00501A75F00A783D30D50508B6FFCF
:1027F7000106C6A426F620D5047002D22780D92464
:10280700CFB41A00EF5004C2E5D228022983D2259B
:1028170080C6D22480C0D22680BCD2D580BAD22925
:1028270080B47F201227722026077401B53D00402F
:10283700F1122737FF1227720227ABD22CD22A8038
:1028470095122737FB122737FA122737F94A4B70A9
:102857000679547A2A7BFF20262EE53D602A7E00E2
:102867008E82758300122C7F60060EEE653E70F037
:10287700C2D5EBC0E0EAC0E0E9C0E0EE1229CAD059
:10288700E0F9D0E0FAD0E0FB122C66FF60AAEBC0BB
:10289700E0EAC0E0E9C0E0122772D0E02401F9D0F5
:1028A700E03400FAD0E0FBE53E0460DCD53ED98099
:1028B700877BFF7A2979C6D226809C791080027996
:1028C70008C22AC22C8008D2D5790A8004790AC2A4
:1028D700D5E53E047002F53EE4FAFDFEFF12273708
:1028E700FC7B08202513122737FD7B1030240A12A2
:1028F7002737FE122737FF7B20EC3382D592D5503E
:1029070013C3E43024069FFFE49EFEE42025039DC5
:10291700FDE49CFCE4CBF8C225EC700CCFCECDCC0B
:10292700E824F8F870F38017C3EF33FFEE33FEEDBA
:1029370033FDEC33FCEB33FB994002FB0FD8E9EB9B
:10294700302505F8D0E0C448B225C0E00AEC4D4E6A
:102957004F78207B0070C2EAB53E0040BCC0E01251
:1029670029CCD0F0D0E0202504C4C0E0C4B225C0F3
:10297700F012275BD0F0D5F0EB0227AB122D6C28B5
:10298700485328C25828194C28154228C64F28CE24
:0F2997004428CE49282E4328D45528B84628B8BE
:1029A6004528B8472A7450281D2D28212E28442B47
:1029B6002825232842202A5D2A27DD480000283CB6
:1029C6003F3F3F00790AA2D5202714302909B910C4
:1029D600020404B9080104A2D5202A0250010420E9
:1029E60026689226B53D005034C0E07F2030271976
:1029F6007F30A226722A7229500F122A23C226C2BB
:102A06002AC229C22C7F30800F302903E9C0E01288
:102A16002772302903D0E0F9D0E0B53DCC30291734
:102A26007F30B9100C1227727F583028077F7880C4
:102A360003B908031227723026057F2D0227727FFD
:102A460020202CF87F2B202AF322922680CF286E76
:102A5600756C6C2900D2251227373025F8C22578E7
:102A66003D30D50108F60227DD2D5043495812277F
:102A7600372403B405004001E4902A6F93122763BC
:0D2A8600743A122763D227753D040228C25E
:10392B008B288A29892AE4F534F533F532F531F5FC
:10393B002FF530E52C452D452B6012EBC0E0EAC08E
:10394B00E0E9C0E0AB2BAA2CA92D122D1DAB28054D
:10395B002AE52AAA297002052914F9122C66F535D5
:10396B00C394094007E535D3940D40E1E535642058
:10397B0060DBE535B42D054330038016E535B42BFC
:10398B0005433001800C74FF252AF52A74FF352975
:10399B00F529E52E60046410703FAB28AA29A92AEB
:1039AB00122C6664306009E52E702E752E0A802964
:1039BB00900001122C7FFF64786004EFB45813431E
:1039CB003001752E107402252AF52AE43529F529C4
:1039DB008007E52E7003752E08AB28052AE52AAA69
:1039EB00297002052914F9122C66F535C394614030
:1039FB000AE535D3947A50035335DF74D02535F56A
:103A0B0035C3940A400CE5359411406D74F9253596
:103A1B00F535E535D3952E50604330018534398526
:103A2B003338853237853136AF2E7E00E4FCFDAB63
:103A3B0034AA33A932A831122CBEC8ECC8C9EDC9BF
:103A4B00CAEECACBEFCBE4FCFDFEEB2535F534EE2D
:103A5B003AF533ED39F532EC38F531AF34AE33ADF1
:103A6B0032FCAB39AA38A937A836D3122BEC50034A
:103A7B000239E44330040239E4E53020E003E4800A
:103A8B002DE52C452D452B601EAB28E52A24FFF98F
:103A9B00E52934FFFAEBC0E0EAC0E0E9C0E0AB2B6C
:103AAB00AA2CA92D122D1DE53030E20774FFFFFE65
:103ABB00FDFC22E530AF34AE33AD32AC3130E10337
:043ACB00022BC822E0
:102C6600BB010689828A83E0225002E722BBFE026C
:092C7600E32289828A83E493229F
:102C7F00BB010CE58229F582E5833AF583E022500A
:102C8F0006E92582F8E622BBFE06E92582F8E22254
:0D2C9F00E58229F582E5833AF583E493226E
:102CAC00BB010689828A83F0225002F722BBFE0107
:022CBC00F32201
:102CBE00E88FF0A4CC8BF0A42CFCE98EF0A42CFCB5
:102CCE008AF0EDA42CFCEA8EF0A4CDA8F08BF0A433
:102CDE002DCC3825F0FDE98FF0A42CCD35F0FCEB92
:102CEE008EF0A4FEA9F0EB8FF0A4CFC5F02ECD3957
:0F2CFE00FEE43CFCEAA42DCE35F0FDE43CFC22C4
:102D0D00FAE6FB0808E6F925F0F618E6CA3AF622C7
:102D1D00BB011A89828A83D0F0D0E0F8D0E0F9D0D7
:102D2D00E0FAD0E0FBE8C0E0C0F0022D9B5016E9C0
:102D3D00F8D083D082D0E0F9D0E0FAD0E0FBC082A9
:102D4D00C083022D92BBFE16E9F8D083D082D0E06D
:0F2D5D00F9D0E0FAD0E0FBC082C083022DA4229F
:102D6C00D083D082F8E4937012740193700DA3A3F6
:102D7C0093F8740193F5828883E47374029368600A
:062D8C00EFA3A3A380DF0A
:092D9200EBF608EAF608E9F62266
:092D9B00EBF0A3EAF0A3E9F02239
:092DA400EBF208EAF208E9F22260
:00000001FF
